:100000000C9408050C944F050C944F050C944F0567
:100010000C944F050C944F050C944F050C944F0510
:100020000C944F050C944F050C94BD2C0C94912D01
:100030000C94E1230C944F050C944F050C944F0540
:100040000C944F050C944F050C944F050C944F05E0
:100050000C944F050C942C240C944F050C944F05D4
:100060000C944F050C944F050C944F050C944F05C0
:100070000C944F050C944F050C944F050C944F05B0
:100080000C944F050C944F050C944F050C944F05A0
:100090000C944F050C944F050C944F050C944F0590
:1000A0000C944F050C944F050C944F05C800BE00EE
:1000B000B40000000014BFFFF0FF000000000014B7
:1000C00080FFF0FF0000000000140AFFF0FF0000B6
:1000D0000000165C1E001F002000210022002300EB
:1000E00024002500260027002D002E0000002A00F5
:1000F0004A002B00000014001A0008001500170029
:100100001C0018000C00120013002F0030003100FA
:100110004B001459000004001600070009000A00F3
:100120000B000D000E000F0033003400280000000B
:100130004E00E10000001D001B0006001900050034
:10014000110010003600370038000000E5005200B2
:100150004D00E000E3000000E200000000002C0081
:100160000000000000000057E600E40050005100CD
:100170004F0035003A003B003C003D003E003F0090
:1001800040004100420043004400450000004C0094
:100190004C0001000000010001000100010001000D
:1001A00001000100520001000100010001002A5D70
:1001B00049000100000001000100010001000100F0
:1001C0000100010001000100010001000100000028
:1001D00046000100000001000100010001000100D3
:1001E0000100010001000100AE000000E500A900CF
:1001F000A800010001000000010000000000010053
:10020000000000000000010001000100CA5CAA001B
:10021000C95C290029000000000000000000000067
:1002200000000000000000000000000000000000CE
:100230000000000000002B05F500F000F4000000B5
:100240000000F900000000000000000000000000B5
:100250000000000000005108F200F100F30000006F
:100260000000FB00FC000000000000000000000097
:100270000000285D000000002900000000000000D0
:100280000000FA000000000000000000E50000008F
:100290000000E00000000000E20000000000295D16
:1002A0000000000000000253E600E400000000002F
:1002B000000044454255473A2064697361626C65A9
:1002C000642E0A0044454255473A20656E61626CCF
:1002D00065642E0A000A002530313662003A20009B
:1002E00025303258000A722F6320303132333435D2
:1002F000363738394142434445460A007267626CDA
:10030000696768742073657420687376205B4E4F4C
:10031000454550524F4D5D3A2025752C25752C25AD
:10032000750A007267626C6967687420736574206F
:10033000687376205B454550524F4D5D3A202575D8
:100340002C25752C25750A007267626C69676874C4
:100350002064697361626C65205B4E4F4545505265
:100360004F4D5D3A207267626C696768745F636FB6
:100370006E6669672E656E61626C65203D2025752D
:100380000A007267626C69676874206469736162ED
:100390006C65205B454550524F4D5D3A2072676257
:1003A0006C696768745F636F6E6669672E656E61FE
:1003B000626C65203D2025750A007267626C696772
:1003C000687420656E61626C65205B4E4F454550D8
:1003D000524F4D5D3A207267626C696768745F6363
:1003E0006F6E6669672E656E61626C65203D2025C3
:1003F000750A007267626C6967687420656E616275
:100400006C65205B454550524F4D5D3A20726762E6
:100410006C696768745F636F6E6669672E656E618D
:10042000626C65203D2025750A007267626C696701
:10043000687420746F67676C65205B454550524F48
:100440004D5D3A207267626C696768745F636F6EB6
:100450006669672E656E61626C65203D2025750AB0
:10046000007267626C69676874206D6F6465205BF9
:100470004E4F454550524F4D5D3A2025750A00724A
:1004800067626C69676874206D6F6465205B4545C1
:1004900050524F4D5D3A2025750A007267626C69B3
:1004A0006768745F696E6974207267626C696768F7
:1004B000745F636F6E6669672E6D6F6465203D20A3
:1004C000302E2057726974652064656661756C749E
:1004D0002076616C75657320746F20454550524FCE
:1004E0004D2E0A007267626C696768745F696E6995
:1004F00074206565636F6E666967206973206E6F2F
:100500007420656E61626C65642E0A007267626CAD
:10051000696768745F696E697420737461727421AD
:100520000A007267626C696768745F696E6974203B
:1005300063616C6C65642E0A007267626C6967683F
:10054000745F636F6E6669672E7370656564203DC6
:100550002025640A007267626C696768745F636F64
:100560006E6669672E76616C203D2025640A0072F4
:1005700067626C696768745F636F6E6669672E7324
:100580006174203D2025640A007267626C696768A7
:10059000745F636F6E6669672E687565203D202500
:1005A000640A007267686C696768745F636F6E667F
:1005B00069672E6D6F6465203D2025640A007267AF
:1005C000626C696768745F636F6E6669672E656EDB
:1005D00061626C65203D2025640A007267626C6967
:1005E0006768745F636F6E66696720454550524F58
:1005F0004D3A0A006261636B6C69676874207374BA
:1006000065703A2025750A006261636B6C696768E2
:10061000742064697361626C650A006261636B6C6B
:100620006967687420656E61626C650A0062616367
:100630006B6C6967687420746F67676C653A202516
:10064000750A006261636B6C696768742064656336
:1006500072656173653A2025750A006261636B6C8F
:100660006967687420696E6372656173653A2025F5
:10067000750A0000010101010101010101020202EC
:10068000020202020202030303030303030304043E
:100690000404040404050505050506060606060708
:1006A0000707070708080808090909090A0A0A0BC1
:1006B0000B0B0C0C0C0D0D0D0E0E0E0F0F0F101062
:1006C00011111112121313141415151616171718E9
:1006D0001819191A1A1B1B1C1D1D1E1E1F20202154
:1006E0002222232424252626272829292A2B2C2D9B
:1006F0002D2E2F30313232333435363738393A3BBC
:100700003C3D3E3F404142434445464748494A4CB0
:100710004D4E4F50515354555658595A5B5D5E5F7C
:10072000616264656668696B6C6D6F707273757712
:10073000787A7B7D7E8082838587888A8C8E8F9174
:10074000939596989A9C9EA0A2A3A5A7A9ABADAF9E
:10075000B1B3B5B7BABCBEC0C2C4C6C9CBCDCFD188
:10076000D4D6D8DBDDDFE2E4E7E9EBEEF0F3F5F831
:10077000FAFDFF0A002530325820006B6579626F60
:100780006172645F7265706F72743A20000A0025AE
:10079000303258006B6579626F6172645F736574A3
:1007A0005F6C65643A200064656C5F6B65795F62BD
:1007B00069743A2063616E27742064656C3A202561
:1007C0003032580A006164645F6B65795F626974F6
:1007D0003A2063616E2774206164643A20253032C8
:1007E000580A00290A002575002F002575005D288C
:1007F00000256400200025640020002564002000FE
:100800002564007C0025303258006D6F7573656B70
:100810006579205B62746E7C782079207620685D33
:10082000287265702F61636C293A205B005B735DF1
:10083000004B6579626F6172642073746172742E0B
:100840000A005B575D005B535D005B525D005B44DB
:100850005D005B435D0004033000000010034B00AB
:1008600042004400360037007600320000001003DA
:100870004B0042004400460061006E00730000001F
:100880000403090409025B00030100A0FA09040043
:1008900000010301010009211101000122400007AC
:1008A00005810308000A0904010001030000000992
:1008B000211101000122BC000705820320000A0962
:1008C000040200020300000009211101000122229C
:1008D0000007058303200001070503032000011220
:1008E00001100100000008424B6760020001020392
:1008F000010631FF0974A1010975150026FF009555
:1009000020750881020976150026FF0095207508DC
:100910009102C005010902A10185020901A100059A
:100920000919012905150025019505750181029513
:1009300001750381010501093009311581257F9574
:10094000027508810609381581257F950175088192
:1009500006050C0A38021581257F95017508810668
:10096000C0C005010980A101850319012AB700153E
:100970000126B700950175108100C0050C0901A181
:1009800001850419012AA002150126A0029501750E
:10099000108100C005010906A1018505050719E0C0
:1009A00029E7150025019508750181020507190041
:1009B00029EF1500250195F075018102050819013F
:1009C0002905950575019102950175039101C005F1
:1009D000010906A101050719E029E7150025019580
:1009E0000875018102950175088101050719002923
:1009F000FF150026FF0095067508810005081901FE
:100A00002905950575019102950175039101C000B5
:100A100011241FBECFEFDAE0DEBFCDBF04B603FE68
:100A200027C08091160390911703A0911803B091ED
:100A300019038730904BA740B04BD1F410921603A6
:100A400010921703109218031092190314BE84B762
:100A5000877F84BF0FB6F894A89580916000886165
:100A600080936000109260000FBEE0E0F8E309950B
:100A700011E0A0E0B1E0EEEAF0E602C005900D92D0
:100A8000AC3BB107D9F723E0ACEBB1E001C01D925C
:100A9000A631B207E1F70E94F2290C9419300C94A8
:100AA0000000FF93EF93E091BC01F091BD013097FE
:100AB00009F00995EF91FF910895FC01859180302F
:100AC00011F0EFDFFBCF0895FF27E0E230E247FFB0
:100AD0000CC0419597FF09C0EDE260957095809537
:100AE0009095611D711D811D911D27FF02C02195EB
:100AF00030E350E2AA27660F771F881F991FAA1FAD
:100B0000A41710F0A41B63955A95A9F7AA3008F012
:100B1000A95FA05DAF93F3956115710581059105FE
:100B200041F7ED3211F4EF93F395F21718F43F9378
:100B3000F395FBCF8F91B5DFFA95E1F70895E99131
:100B4000F9918591803021F0853219F0AADFF9CF33
:100B5000089520E0E89455915532C1F3503311F4D3
:100B6000689455915A3348F4505390F3220F022E53
:100B7000220F220F200D250FF4CF0EF4219589911D
:100B80009991533619F3533729F1533559F1BC0173
:100B900088279927E8945C3621F489919991689483
:100BA0005591543639F446EF7EF077FF0DC08FEF44
:100BB0009FEF0AC055374AE039F0583540E121F03F
:100BC000523642E009F00895FF93EF937DDFEF91F5
:100BD000FF91B7CFFF93EF93FC0181918030B9F380
:100BE00060DFFBCFFF93EF9368DFF1CFDF93CF930D
:100BF000CDB7DEB72596A3DFCF91DF910895549A44
:100C00000C945106CF93C82F0E948607882319F0B1
:100C1000C1FD03C05C9ACF9108955C98FCCF809190
:100C20000101823019F481E00E94A11F109201019C
:100C300008958091BE018F5F833018F48093BE01C8
:100C400008951092BE0108958CEA90E09093C3013C
:100C50008093C2010895CF92DF92EF92FF926B01D1
:100C60007C0140E00E944B1F682F80E00E940C1026
:100C700041E0C701B6010E944B1F682F81E00E942E
:100C80000C1042E0C701B6010E944B1F682F82E0A2
:100C90000E940C10C701B601FF90EF90DF90CF903B
:100CA000089508950895CF93DF93EB0189322DE5E0
:100CB000920799F18A322DE59207A1F188329D457C
:100CC000C9F5CA818091BE01CC23B1F0813071F0A9
:100CD000882339F0823069F0C0E08C2FDF91CF910A
:100CE00008958DEF90E00E94FB06F6CF8EEF90E026
:100CF000FACF8FEF90E0F7CF813061F0882329F0B1
:100D0000823059F78FEF90E002C08DEF90E00E94A3
:100D10001007E3CF8EEF90E0FACF8A81811102C0F5
:100D20000E941906CA81CC2329F00E94060E0E9457
:100D30009107D3CFC1E0D1CFFC018081813029F46C
:100D40009285992339F082E00895823011F088E08D
:100D5000089583E008950E949C06809301018823F2
:100D600091F0833018F0833021F0089581E00C94E5
:100D7000801F82E00E94601F882319F082E00C949B
:100D8000A11F82E0F4CF0895CF93DF939C013A95A1
:100D900021153F4168F5EC01CC27D170DC01AA2771
:100DA000B270AC01442754709C012227387094FF24
:100DB00011C080E1CD2B09F480E0AB2B09F08062FB
:100DC000452B09F08064232B09F08068FB01DF913B
:100DD000CF91099481E0CD2B09F480E0AB2B09F091
:100DE0008260452B09F08460232B81F38860EECF6D
:100DF000DF91CF910895CF93DF93EC01805E91094D
:100E0000089720F061E47BE1209711F46BED78E125
:100E1000CE010E94C4068C2FDF91CF910C94E01775
:100E2000CF93DF93EC010E947218CE01805E91098E
:100E3000089720F068E47BE1209711F462EE78E1F6
:100E4000CE01DF91CF910C94C40681E008950C94FB
:100E5000530608950C9429071F93CF93DF9300D076
:100E600000D00F92CDB7DEB749835A836B833091A0
:100E7000DF0189819A8131111DC06623B9F02223D7
:100E8000A9F00E946F20182F682F89819A810E94F3
:100E90001C2069817A81812F0F900F900F900F9005
:100EA0000F90DF91CF911F910C940C080E94482065
:100EB000182FEFCF0E946F2069817A81EDCFFC015E
:100EC000262F408151816281738184810C942C078B
:100ED000CF93DF93EC0160E00E945F07BE01DF91DA
:100EE000CF910C942A070E9476240E94E62181115A
:100EF00002C00E948C220E944F120C94FF050E9497
:100F0000BA150C94180A08950C94830781E008958B
:100F1000CF93C82F0E9484078C2FCF910C94020688
:100F200008950E94651B0E9490072FEF84E39CE0C8
:100F3000215080409040E1F700C000000C94502404
:100F40000F931F93CF93DF93EC0161E00E945F0743
:100F50008C01BE010E941A15BE01C8010E9427071C
:100F60008823A1F1BE01C8010E94BB11882371F141
:100F7000BE01C8010E946015882341F1BE01C8016D
:100F80000E941613882311F1BE01C8010E94681344
:100F90008823E1F0BE01C8010E948B148823B1F0C0
:100FA000BE01C8010E942E10882381F08A81882307
:100FB00041F101308CE5180779F00E3D8CE51807FA
:100FC000E9F001151C45E9F40E94910780E0DF91EA
:100FD000CF911F910F91089590917702892F8E7F65
:100FE00090FF81608093770280FF05C084EC92E0DF
:100FF0000E945D05EBCF82EB92E0FACF0E948C223B
:10100000E5CFCE01DF91CF911F910F910C94250771
:1010100090E080E008950895E72FF0E095E0899F43
:10102000E00DF11D112484E0EE0FFF1F8A95E1F71A
:10103000E60FF11DEE0FFF1FEE52FF4F85919491C9
:101040000895FC01EE0FFF1FEB52FD4F8591949127
:101050000895CF93DF930E940C080E943E09EC0193
:10106000811520E5920708F042C0811530E493070E
:1010700008F0BDC0883E910528F5803E910508F036
:101080009DC0883A910588F4853A910508F08FC093
:101090008130910509F492C0009709F48FC004973C
:1010A00008F08CC0D0E0C0E089C08F3B910508F407
:1010B00089C0805C9109C03CD105A0F30E94210841
:1010C000EC017CC08115904250F4C11581E0D80735
:1010D00008F074C0C03FD10528F3D0656FC0C115BA
:1010E00090E3D90708F079C0CE019F70E7CF811552
:1010F00025E5920758F5811534E5930708F0A6C059
:10110000811542E5940750F4C11581E5D80708F42C
:1011100071C0DC2FCC27C16FD06A50C0982F969534
:1011200096959E0123703327C115D34508F07FC0E3
:10113000C1E0D0E002C0CC0FDD1F2A95E2F720E22B
:10114000929FC0011124C82BD92B6FC0C11589E50E
:10115000D807A8F4C11598E5D90708F07CC0C115D7
:1011600026E5D20708F09ECF8C2F0E94D509C82F04
:10117000D0E0DC2FCC27CC27DF71D0621FC0C11597
:101180003AE5D30708F46CC0CE0190568115904221
:1011900008F088CF8D2F8F710E94D50990E0982F8D
:1011A000882788279F719C012C2BE901E6CFC55A1F
:1011B000D0E0CF59DE4FC881D0E0D064CE01DF91BE
:1011C000CF910895C85AD0E0CC0FDD1FCD5CDE4F23
:1011D0000990D881C02DD464F1CFCE019927D3FFD7
:1011E00003C0EC01D86CEACFEC01D06CE7CFDF7024
:1011F000D06AE4CFCE01E4E096958795EA95E1F7D1
:1012000083702C2F26952695237090E2299F9001BC
:101210001124382B8C2F8370C1E0D0E002C0CC0F9A
:10122000DD1F8A95E2F7C22BD32BDC68C7CFC1E064
:10123000D0E002C0CC0FDD1F2A95E2F730E2939F89
:10124000C0011124C82BD92BDA68B8CFD82FCC27EE
:10125000C46FD06AB3CFDC2FCC27C06FD06AAECFBB
:101260008C2F8F700E94D50934E0D695C7953A959A
:10127000E1F7CF709C2FEC01D069A0CF82389105A7
:10128000B1F1B0F48133910509F475C048F48932A5
:10129000910509F469C08A32910509F473C0089573
:1012A0008533910509F459C08933910501F10895F9
:1012B000833E9105A9F138F4803E9105F9F0823E14
:1012C000910549F10895863E9105A9F1873E910562
:1012D000C9F1843E910519F52091AE0221FF1FC08E
:1012E0008091AD0284FD14C087EE90E008952091B6
:1012F000AD022370A1F080EE90E008952091AD0240
:1013000020FD47C03091AE0230FF09C024FF44C029
:1013100090E080E004C02091AD0222FDF7CF089557
:101320002091AD0222FD3BC03091AE0230FDE3CFF3
:1013300024FFF5CFEDCF2091AD0223FFF0CF24FDA8
:10134000E7CFD2CF2091AD0223FD2CC03091AE0269
:1013500031FFEECF84EE90E008952091AD0225FF9D
:10136000DECF89E290E008952091AD0225FFD7CF2E
:1013700085E390E008952091AD0226FFD0CF8AE268
:1013800090E008952091AD0226FFC9CF81E390E05F
:10139000089589E390E0089583EE90E0089582EE49
:1013A00090E0089586EE90E008959091AD0292FF4E
:1013B00006C0282F28712830F9F4877F846093FFB6
:1013C00006C0282F28712831F1F4877E846120918E
:1013D000AE0220FF06C0382F38713830D9F4877F2D
:1013E000816021FF06C0282F28712831D1F4877E23
:1013F000816194FD877E0895282F24712430F9F6A9
:101400008B7F8860DCCF282F2471243101F78B7EFD
:101410008861DDCF382F3171313019F78E7F8860C8
:10142000E0CF282F2171213121F78E7E8861E1CF15
:101430000C945206E82FF0E0EE0FFF1FE754FD4F2B
:10144000808191810895CF92DF92EF92FF920F9366
:101450001F93CF93DF9385EE92E00E945D0589EBA9
:10146000E82E82E0F82ED0E0C0E090EEC92E92E0A7
:10147000D92E07ED12E0DF93CF93DF92CF920E9437
:10148000F6058DED92E00E945D05F7018191919145
:101490007F010E94D3219F938F931F930F930E94EC
:1014A000F60585ED92E00E945D0521968DB79EB709
:1014B00008960FB6F8949EBF0FBE8DBFC530D105FC
:1014C000D1F6DF91CF911F910F91FF90EF90DF90B8
:1014D000CF90089580EA8A95F1F70895CF93DF932E
:1014E000A4E7B1E049E751E0C1E0D0E08D91E82FF9
:1014F000E295EF70F0E061A18F709E0101C0220FB4
:101500008A95EAF7922F9095962391A382A1822B38
:1015100082A34A175B0751F7A4E6B1E061E070E0EF
:101520008D91E82FE295EF70F0E041A18F709B0163
:1015300001C0220F8A95EAF7922F9095942391A3E8
:1015400082A1822B82A381E0A437B80749F71092C9
:10155000B0021092AF021092BA021092B902109229
:10156000B2021092B1021092BC021092BB02109211
:10157000B4021092B3021092BE021092BD021092F9
:10158000B6021092B5021092C0021092BF021092E1
:10159000B8021092B7021092C2021092C10285E006
:1015A0000E945D0BDF91CF910C9473078F929F92F5
:1015B000AF92BF92CF92DF92EF92FF920F931F9361
:1015C000CF93DF9384E7E82E81E0F82E0FEA12E054
:1015D000912CAA24A394B12CF70181917F01C82FEB
:1015E000C295CF70D0E099A18F70650101C0CC0C7D
:1015F0008A95EAF7892F8C2989A38AA18C2C80945B
:1016000088218AA30E946A0AE4E6F1E050E040E003
:1016100030E020E06191A62FA295AF70B0E09096E7
:101620008C9190E06F7002C0959587956A95E2F76E
:1016300080FD3EC0C501042E02C0880F991F0A9488
:10164000E2F7282B392B4F5F5F4F4031510511F7DF
:1016500089A1882289A28AA1C82ACAA2F801808108
:1016600091812817390739F13183208381E0982A45
:101670000E5F1F4FF9E7EF16F1E0FF0609F0ACCF60
:10168000292D45E069EB72E08FEA92E00E945E0B43
:101690000E947F07892DDF91CF911F910F91FF90BD
:1016A000EF90DF90CF90BF90AF909F908F90089574
:1016B00090E080E0C6CF80E0DACF0895FF920F93EC
:1016C0001F93CF93DF93F82E092F162FD72FC42FF8
:1016D000222349F081E08093C1010E94112490935C
:1016E000C0018093BF018091C1018823A1F0809146
:1016F000BF019091C0010E941D24069760F0EF2D5C
:10170000F02FA12FBD2F90E080E0D0E08C179D0737
:1017100044F01092C101DF91CF911F910F91FF9082
:101720000895219131912D933D930196EFCFEF9242
:10173000FF920F931F93CF93DF93EB01E82FD1110B
:1017400010C0442321F0F0E0ED58F94FE4916E2FE2
:101750007E2F8E2FDF91CF911F910F91FF90EF90F1
:1017600008950D2F10E0282F30E0442329F02D5844
:10177000394FF901249130E0F6E0CF9FC0011124E8
:10178000EFEFF0E0BF010E945E2FAB018C2F90E0E5
:10179000880F991FA5E5A49FB001A59F700D112486
:1017A000861B970B982F990F980FBF01601B710B29
:1017B000629FD001639FB00D729FB00D11248B2FDB
:1017C0009D9FB0011124672F7727EF01C61BD70B10
:1017D000BE01629FE001639FD00D729FD00D112466
:1017E0007F01E91AF108E09EB001E19E700DF09EC4
:1017F000700D1124672F7727E61BF70BE29F8001FE
:10180000E39F100DF29F100D1124E12F722F423033
:10181000510599F048F44115510569F041305105E1
:1018200081F0EB2F8D2F07C04430510569F080F017
:1018300046305105B1F76E2F8DCFE22F7B2F812FD0
:10184000FACFE22F7D2FF7CFEB2F822F712FF3CF1F
:101850007B2F822FED2FEFCF41E00C94970BCF938E
:10186000DF93762FE901682F842F0E942C0C798357
:1018700068838A83DF91CF910895413F08F040EF5C
:101880000C942F0C8091C302982F9E7F71F480914D
:10189000C302817082608093C3028091C602813F3F
:1018A00018F080EF8093C6020895843080F7F5CF5A
:1018B00088E090E00C94D92FCF92DF92EF92FF92C4
:1018C0006B017C010E94420CB701A60188E090E008
:1018D000FF90EF90DF90CF900C94F72FE3ECF2E0C5
:1018E00083E0808311828FEF828380EF8383148271
:1018F00060817181828193810C945C0C809177026C
:1019000080FF76C08BED95E09F938F930E94F60544
:10191000809177020F900F9080FF6AC08091C30280
:1019200081701F928F938EEB95E09F938F930E940F
:10193000F605809177020F900F900F900F9080FF27
:1019400057C08091C30286951F928F9383EA95E0DA
:101950009F938F930E94F605809177020F900F90CE
:101960000F900F9080FF44C08091C4021F928F930C
:1019700089E895E09F938F930E94F6058091770206
:101980000F900F900F900F9080FF32C08091C50292
:101990001F928F938FE695E09F938F930E94F60599
:1019A000809177020F900F900F900F9080FF20C0D2
:1019B0008091C6021F928F9385E595E09F938F9348
:1019C0000E94F605809177020F900F900F900F9074
:1019D00080FF0EC08091C7021F928F9389E395E02C
:1019E0009F938F930E94F6050F900F900F900F908A
:1019F00008959091C702933018F49F5F9093C702A7
:101A0000882351F06091C3027091C4028091C50295
:101A10009091C6020C945C0C089581E00C94F90C32
:101A20009091C702992319F091509093C70288238F
:101A300051F06091C3027091C4028091C5029091EF
:101A4000C6020C945C0C089581E00C94100D21E00A
:101A500030E001C0220F8A95EAF79091C7019223E6
:101A600081E009F480E0089570E00C945F126F92B9
:101A70007F928F929F92AF92BF92CF92DF92EF921E
:101A8000FF920F931F93CF93DF9300D000D00F925C
:101A9000CDB7DEB7709019019091C30290FF26C0B8
:101AA000C090C201D090C301C114D10489F58091C6
:101AB000180133E0839FC0011124672D88539D4F87
:101AC0000E94340D0F900F900F900F900F90DF91A8
:101AD000CF911F910F91FF90EF90DF90CF90BF902B
:101AE000AF909F908F907F906F90089580911A0192
:101AF00020911B0133E0839FF0011124E853FD4F37
:101B0000821770F61182108212828F5F3396F8CF9F
:101B100090FFCDCFF12CE12C43E0642E8E2D0E945E
:101B2000270D882309F43CC0F701EE0FFF1FEC0DD1
:101B3000FD1DA590B490A114B10409F4B8CF45E0FF
:101B400050E0B501CE0101960E94C82F09810F3FD8
:101B500039F18A81800F9927991F8531910514F0F9
:101B600084E190E04C01880C991C880D991D9C0122
:101B700028533D4F4901069D8001112408531D4FF4
:101B80000815190520F035E0A30EB11CD8CF980137
:101B90004D816C818B810E943D0C0D5F1F4FF0CFFA
:101BA0008FEFE81AF80A28E0E216F10409F0B6CF40
:101BB0007ECF8091C3028E7F8093C3026091C30267
:101BC0007091C4028091C5029091C6020E945C0C83
:101BD0008091770280FF0FC08091C30281701F92B5
:101BE0008F9382E893E09F938F930E94F6050F9066
:101BF0000F900F900F902FEF80E792E021508040E0
:101C00009040E1F700C000000C94370D8091C302B2
:101C10008E7F8093C3028091770280FF0CC01F9259
:101C20001F9288E493E09F938F930E94F6050F9094
:101C30000F900F900F902FEF80E792E0215080409F
:101C40009040E1F700C000000C94370D9091C30262
:101C500090FF14C090911A0120911B0133E0939FD3
:101C6000F0011124E853FD4F921710F00C94370D3A
:101C70008183608342839F5F3396F6CF0895EF920E
:101C8000FF920F931F93CF93DF9300D00F92CDB7A6
:101C9000DEB7182F062FF42EE22E8091C30280FFAC
:101CA00043C0E82FE695F0E0E758FE4F908190930F
:101CB000C5018E7F823059F49E012F5F3F4F812FE7
:101CC0000E943D0C4B8169818A810E94260E1093EF
:101CD000C4020093C502F092C602EE2079F1609131
:101CE000C3027091C4028091C5029091C6020E9405
:101CF0005C0C8091770280FF17C08091C6021F9212
:101D00008F938091C5021F928F938091C4021F927E
:101D10008F9383E293E09F938F930E94F6050FB613
:101D2000F894DEBF0FBECDBF0F900F900F90DF91E4
:101D3000CF911F910F91FF90EF90089580917702BE
:101D400080FFF2CF1F92FF921F920F931F921F935B
:101D50008CEF92E0E0CFE3ECF2E09181282F438119
:101D6000628188E0890F0C943F0E81E00C94AB0EE9
:101D7000E3ECF2E09181282F4381628188EF890FA3
:101D80000C943F0E81E00C94B80EE3ECF2E062811B
:101D900028E0620F08F46FEF282F438181810C94B3
:101DA0003F0E81E00C94C50EE3ECF2E0628128E086
:101DB000621B08F460E0282F438181810C943F0E60
:101DC00081E00C94D40EE3ECF2E0438128E0420F72
:101DD00008F44FEF282F628181810C943F0E81E03F
:101DE0000C94E30EE3ECF2E0438128E0421B08F49C
:101DF00040E0282F628181810C943F0E81E00C9499
:101E0000F20E20E00C943F0E8091C30280FF35C09B
:101E1000817082608093C302662329F16091C302BE
:101E20007091C4028091C5029091C6020E945C0C20
:101E30008091770280FF0FC08091C30286951F9228
:101E40008F938FE794E09F938F930E94F6050F90F6
:101E50000F900F900F904091C6026091C502809143
:101E6000C4020C94010F8091770280FFF4CF1F927F
:101E700081E08F9381E694E0E6CF0895682F81E0BA
:101E80000C94040F81E00C943E0F682F9091C302D4
:101E900096958FEF890F09F481E00C94040F81E08F
:101EA0000C94450F61E00C94040F8091C302816093
:101EB0008093C3028091770280FF0DC01F9281E062
:101EC0008F9383EF93E09F938F930E94F6050F907B
:101ED0000F900F900F908091C30286950C94520F33
:101EE0008091770280FF10C08091C302809581703D
:101EF0001F928F938AE294E09F938F930E94F6053E
:101F00000F900F900F900F908091C30280FD0C9462
:101F1000D90D0C94550F60E00C94040F8091C4010E
:101F200081115EC08091770280FF14C082E295E04B
:101F30009F938F930E94F605809177020F900F90E8
:101F400080FF08C08CE095E09F938F930E94F60578
:101F50000F900F900E94E621811110C080917702AE
:101F600080FF08C084EE94E09F938F930E94F60553
:101F70000F900F900E948C220E946E0C0E94580CB1
:101F80006093C3027093C4028093C5029093C6020B
:101F90006E7FC1F48091770280FF08C08BE994E0E6
:101FA0009F938F930E94F6050F900F900E946E0CE6
:101FB0000E94580C6093C3027093C4028093C502C0
:101FC0009093C6020E94420C0E947E0C8091C30234
:101FD00080FF03C086950E948B0F81E08093C4012F
:101FE00008958091C30281608093C302809177023B
:101FF00080FF0DC01F9281E08F938AEB93E09F9347
:102000008F930E94F6050F900F900F900F90809184
:10201000C30286950C948B0F21E030E0A90102C029
:10202000440F551F8A95E2F7CA012091C701662324
:1020300061F0822B8093C7018091C601811108C095
:102040008091C30286950C948B0F80958223F2CFEA
:102050000895FA01811101C0FB0109940F931F93A8
:10206000CF938C01FB01C281CC2309F44DC00E94A7
:1020700004218272F801E25CFC45E431F10538F498
:10208000E55EFF4C0C94A82F0E94700FC0E08C2FCF
:10209000CF911F910F9108954FE45FE062E47FE0DC
:1020A0000E942910F3CF42E45FE06FE47FE0F8CFB5
:1020B00042EC5EE065EB7EE0F3CF45EB5EE062EC88
:1020C0007EE0EECF40EE5EE061ED7EE0E9CF41EDF7
:1020D0005EE060EE7EE0E4CF4EEF5EE06FEE7EE02D
:1020E000DFCF4FEE5EE06EEF7EE0DACF44E25DE000
:1020F0006DE07DE0D5CF4DE05DE064E27DE0D0CFE6
:1021000081E00E94520FC2CFC1E0C1CF0E94E62100
:10211000811102C00E948C220E9414228093040329
:10212000803220F0877088618093040390910403CB
:10213000892F817090FF04C0892F8695869586959A
:102140000C94F01180910403982F9695969596958E
:10215000933040F49F5F990F990F990F8770892BE7
:1021600080930403809104038160809304030E94A0
:1021700018228091770280FF11C080910403869518
:10218000869586951F928F938BE596E09F938F930C
:102190000E94F6050F900F900F900F90809104030E
:1021A0008695869586950C94F01180910403982F5E
:1021B000987F79F0885080930403887F91E009F438
:1021C00090E08091040390FB80F9809304030E94C7
:1021D00018228091770280FF11C0809104038695B8
:1021E000869586951F928F9383E496E09F938F93B5
:1021F0000E94F6050F900F900F900F9080910403AE
:102200008695869586950C94F0118091040380FD47
:102210001FC0816080930403813019F489E08093AA
:102220000403809104030E9418228091770280FFAA
:1022300008C08BE196E09F938F930E94F6050F9064
:102240000F90809104038695869586950C94F011E5
:1022500008958091040380FF14C08E7F809304034F
:102260000E9418228091770280FF08C088E096E0E3
:102270009F938F930E94F6050F900F9080E00C942F
:10228000F0110895CF93C0910403C170809177023B
:1022900080FF0CC01F92CF938DE296E09F938F93A7
:1022A0000E94F6050F900F900F900F90CC2319F01D
:1022B000CF910C942911CF910C94051190910403A6
:1022C000892F8695869586958F5F8F71977084305C
:1022D00080F5880F880F880F892B809304038091E5
:1022E0000403887F91E009F490E08091040390FB5F
:1022F00080F9809304030E9418228091770280FF66
:1023000011C0809104038695869586951F928F93C0
:1023100084EF95E09F938F930E94F6050F900F90A6
:102320000F900F90809104038695869586950C9466
:10233000F01190930403D3CF843008F083E09091A0
:1023400004039770282F220F220F220F922B9093B5
:102350000403987F21E009F420E09091040320FB1E
:1023600090F9909304030C94F0110E949C118091B9
:1023700004030C9418229C01FB018281882349F1FB
:102380002D3BFCE53F07C9F040F42B3BECE53E0755
:1023900069F02C3B3C4579F008952F3B9CE53907CB
:1023A00091F070F0203C3C4589F0089583E00E9454
:1023B000B51180E0089580E0FACF0E94D510F9CFE2
:1023C0000E94A210F6CF0E944211F3CF0E945E112C
:1023D000F0CF81E00895259A2D9808952D980895BD
:1023E000CF92DF92EF92FF92CF93C82F843040F5C7
:1023F000811127C0809180008F77809380000E9498
:10240000EE112C2F30E0AFEFBFEF0E94AE2F23E094
:1024100030E040E050E00E94862FC9012C3764E193
:102420003607A8F469E070E00E945E2F709389007F
:1024300060938800CF91FF90EF90DF90CF90089548
:10244000C3E080918000806880938000DACF2A50BA
:10245000374D4F4F5F4F942F832F722F662725EFF5
:1024600038E241E050E00E94862F69017A01CA01FA
:10247000B9010E94422F9B01AC01C701B6010E9425
:10248000422F672F782F892F99276115710521E039
:102490008207910559F66FEF7FEFC8CF08950E942C
:1024A000EB1182E88093800089E1809381008FEFB7
:1024B0009FEF90938700809386000C9486106A9A11
:1024C0004EB14B7F5EB15460EFB7F8949B01220F81
:1024D000331F260F371F280F391F2817390741F4DC
:1024E000EFBF8FE594E00197F1F700C00000089579
:1024F000DC016D91CD0178E05EB9000000C067FF9E
:102500004EB9660F000000C000C000C04EB900C048
:102510007A9591F7E2CFAF92BF92CF92DF92EF928E
:10252000FF920F931F93CF93DF937C015B01C42F26
:10253000D22FFC0182818823F9F04093CA010E94C6
:1025400011249093C9018093C80180E28C0F8830D8
:1025500008F061C0C77081E001C0880FCA95EAF732
:10256000DF91CF911F910F91FF90EF90DF90CF906F
:10257000BF90AF900C94DB181091CA01141340C0A7
:102580008091C8019091C9010E941D246C01B7017E
:10259000C5010E94DB1DC816D90690F5C0E2CD0F1B
:1025A0001D17B9F080E2810F883040F4177081E088
:1025B00001C0880F1A95EAF70E94E218C83048F463
:1025C00081E09D2F977001C0880F9A95EAF70E94CD
:1025D000DB18802F0E94C818C830E8F4D77081E05B
:1025E00001C0880FDA95EAF7DF91CF911F910F9123
:1025F000FF90EF90DF90CF90BF90AF900C94E218D7
:1026000080E28C0F883038F4C77081E001C0880FF9
:10261000CA95EAF7E9CFDF91CF911F910F91FF9013
:10262000EF90DF90CF90BF90AF9008950F939C01F3
:10263000CB01233F4CE5340759F1A8F4283DFCE5D4
:102640003F0701F1293D4CE53407D1F1273D3C45D9
:1026500091F406E221EE41EE67ED7CE50E948B12DB
:1026600080E00F910895253FFCE53F07E9F0B0F0C9
:10267000263F3C45F9F0FC018281882339F1109214
:10268000CA01EFCF07E225EE45EE68ED7CE5E6CF27
:1026900006E221EE40EE63EF7CE5E0CF07E225EEB7
:1026A00044EE64EF7CE5DACF06E221EE42EE65EF20
:1026B0007CE5D4CF07E225EE46EE66EF7CE5CECF93
:1026C00008E221E045EE69ED7CE5C8CF81E0C9CFA5
:1026D000CF93DF93EC01FB018281882309F419C1B8
:1026E000C230FCE5DF07C0F1C6319CE5D90730F008
:1026F0009E012A5F3C452930310570F50E94F92181
:102700009093AE028093AD02C031ECE5DE0709F490
:10271000CFC008F05BC0C8308CE5D80709F4B6C05C
:1027200088F5C430ECE5DE0709F4A8C0C0F4C23077
:102730008CE5D80709F49CC08091AD028260C3305B
:10274000DC4509F498C08091AD029091AE020E94E0
:1027500007220E94651B80E0DF91CF910895809150
:10276000AD028061C630ECE5DE0709F484C08091DB
:10277000AD028860C730DC4508F47DC08091AD02B1
:10278000806279C0CC308CE5D80709F489C070F438
:102790008091AD028C60CA30ECE5DE0709F46BC0B5
:1027A00008F478C08091AD028E7F65C0CE308CE594
:1027B000D80709F479C08091AD028B7FCF30DC451A
:1027C00008F459C08091AD028F7E55C0CB3FECE537
:1027D000DE0709F457C030F5C3318CE5D80709F49A
:1027E0006FC078F4C131ECE5DE0709F465C0C23191
:1027F000DC4509F0A8CF0E94651B8091AD028F7760
:102800003AC0C5318CE5D80709F462C008F476C037
:102810008091AE028160CA3FDC4509F094CF80937D
:10282000AE0291CFCF3FFCE5DF0709F44DC088F43D
:102830008091AE028D7FCD3F9CE5D90781F38091D9
:10284000AE028E7FCE3FDC4550F38091AE028360B6
:10285000E6CFC130FDE5DF0709F459C008F444C0F4
:1028600080E0C230DD4509F06ECF0E948E226BCF32
:102870008091AD0281608093AD0265CF8091AD0201
:102880008460F9CF8091AE028260C9CF8091AD02A1
:102890008064F1CF0E94651B8091AD028068EBCF10
:1028A0008091AD028D7FE7CF8091AD02877FE3CF2E
:1028B0008091AD028F7DDFCF8091AD028F7BDBCF2A
:1028C0008091AD02837FD7CF8091AE028C7FA7CF5E
:1028D0008091AD0282FB992790F921E0922790FB2D
:1028E00082F990FB83F9C7CF8091AE02982F909523
:1028F00091708E7F892B90FB81F991CF0E94651B8F
:102900009091AD02892F97FB87F98058B4CF81E071
:10291000ACCF81E021CFCF93DF93EB0186319C4593
:1029200039F50E940421982F91718A7A911180E0E3
:102930009A81992399F091E0811101C090E09093E0
:10294000CB01811109C089E20E94DF200E9453213E
:1029500080E0DF91CF91089585E3F6CF8091CB01A0
:10296000811104C089E20E94E620F0CF85E3FBCF0D
:1029700081E0EFCFCF93DF93EC0181E0898B8F81F2
:102980000E94072188850E941A210E945321EA8112
:10299000FB81309739F06C897D89CE010696DF91F5
:1029A000CF910994DF91CF910895EF92FF920F9309
:1029B0001F93CF93DF93EC018A85811134C0EB80A4
:1029C000FC8087E5F81A26E12E9DC0012F9D900D11
:1029D0001124DC01AE5FBE4F1496ED91FC9115976A
:1029E000309731F054966D917C91885F9E4F099598
:1029F00086E18E9D80018F9D100D11240E5F1E4F6C
:102A0000F80187810E940D21F80180850E94202114
:102A10000E945321188219861B861E821D821092E5
:102A2000CD011092CC01DF91CF911F910F91FF90BA
:102A3000EF900895DF92EF92FF920F931F93CF9341
:102A4000DF937C01FB018281882391F080911D013D
:102A50008F3F71F0C2E0D1E010E000E0DD24D394BC
:102A600080911D01082E000C990B8017910744F4EA
:102A7000DF91CF911F910F91FF90EF90DF9008951C
:102A80008E818823C9F089859A858E159F0539F432
:102A90008091CC019091CD018E159F0569F0DF8664
:102AA000FC86EB868989811103C0CE010E94BA148D
:102AB000CE0106960E94D5140F5F1F4F6696D0CFA9
:102AC000EF92FF920F931F93CF93DF937C01975563
:102AD0008F3F910509F0D8F520911D01022E000CC1
:102AE000330B2817390714F480931D01FB01228151
:102AF00036E1389F8001399F100D1124E801CE5F27
:102B0000DE4F288B92818E81992349F1FA86E986DE
:102B10008F5F8E830E9411249E878D870E943A21A9
:102B20008F830E94042188870E9417219885892B12
:102B30008887E881F981309731F06C897D89C801F7
:102B4000885F9E4F0995F092CD01E092CC0181E023
:102B5000DF91CF911F910F91FF90EF9008958823FF
:102B6000B1F38989882399F3C801885F9E4F0E9439
:102B7000D514EDCFCF92DF92EF92FF920F931F9378
:102B8000CF93DF9380911D0110E006E18F3FF1F5B7
:102B9000DF91CF911F910F91FF90EF90DF90CF9039
:102BA00008950E9DF0010F9DF00D1124EE5FFE4F74
:102BB000C288D388C114D10439F470E060E0818503
:102BC00092850E94DB1D6C010E9DE0010F9DD00DD2
:102BD0001124CE5FDE4F8E818823B9F08D859E85CE
:102BE0000E941D24C816D90680F4109F700111247C
:102BF0008989811105C0C7018E5F9E4F0E94BA145A
:102C0000C701885F9E4F0E94D5141F5FE12EF12CF3
:102C100080911D01082E000C990B8E159F050CF656
:102C2000B7CF9093D3018093D2010895E091D20160
:102C3000F091D301309721F00190F081E02D0994BB
:102C400080E00895EF92FF920F931F93CF93DF934D
:102C5000EC01E091D201F091D301309709F446C024
:102C600080913201882341F08091AD0287FF04C03A
:102C70008881898385E088830280F381E02DCE01FD
:102C800009958091770282FF31C080FF04C08BE7F5
:102C900097E00E945D0510E000E085E7E82E87E000
:102CA000F82E8091770280FF0EC0FE01E00FF11F29
:102CB00080811F928F93FF92EF920E94F6050F90F2
:102CC0000F900F900F900F5F1F4F0830110549F7BD
:102CD0008091770280FF0AC083E797E0DF91CF9170
:102CE0001F910F91FF90EF900C945D05DF91CF91B4
:102CF0001F910F91FF90EF900895E091D201F09114
:102D0000D301309739F022E0DC012C930480F58167
:102D1000E02D099408952091D0013091D101281718
:102D2000390771F09093D1018093D001E091D201E5
:102D3000F091D301309721F00680F781E02D0994BE
:102D400008952091CE013091CF012817390771F0F5
:102D50009093CF018093CE01E091D201F091D30105
:102D6000309721F00084F185E02D0994089585B70E
:102D7000806885BF85B7806885BF089508950895E8
:102D80000C94BE160C9424060E94B7160E94BF161F
:102D90000C94C01681E008950C94CA160E94082471
:102DA0000E946E0A0E948A240E9486100E948E0F42
:102DB0000C94C216CF93C82F8091770282FF1EC059
:102DC00080FF1CC084E997E00E945D058091770236
:102DD00080FF14C01F92CF938FE897E09F938F934B
:102DE0000E94F605809177020F900F900F900F9040
:102DF00080FF04C08DE897E00E945D058C2FCF9185
:102E00000C9488079F92AF92BF92CF92DF92EF927D
:102E1000FF920F931F93CF93DF93CDB7DEB72A971F
:102E20000FB6F894DEBF0FBECDBF0E94D60A0E9437
:102E3000CC16882309F472C055EDA52E51E0B52EAD
:102E400010E000E0902E802F0E941A0A6C01F5011C
:102E5000E190F1905F01E816F90609F459C08091FC
:102E6000770281FD0E94230A97012C253D2580E0F1
:102E7000EE24E394F12CA9014E215F21452B09F4A6
:102E800041C08E839F82CE20DF2081E0CD2809F4CF
:102E900080E088870E9411248160782F9A87898733
:102EA0004E815F8168858A850E94B117000F111FCE
:102EB000F801EB52FE4F80819181E826F926F182DC
:102EC000E0820E944E120E94A9260E94161690913E
:102ED000D4018917A1F10E9416168093D4012A9675
:102EE0000FB6F894DEBF0FBECDBFDF91CF911F911B
:102EF0000F91FF90EF90DF90CF90BF90AF909F9099
:102F00000C94DA168F5FEE0CFF1C803109F0B3CF02
:102F10000F5F1F4F0530110509F094CF8FEF8983A4
:102F20008A831B820E9411248160782F9D838C8369
:102F300049815A816B818D810E94B117C2CF2A9637
:102F40000FB6F894DEBF0FBECDBFDF91CF911F91BA
:102F50000F91FF90EF90DF90CF90BF90AF909F9038
:102F60000895CF93DF93CDB7DEB72B970FB6F894C4
:102F7000DEBF0FBECDBF4F83588769877A878B87A7
:102F80001E821D8285E0FE013796DE0111960190BA
:102F90000D928A95E1F749815A816B817C818D81FF
:102FA0009E812B960FB6F894DEBF0FBECDBFDF918A
:102FB000CF910C94DE1DFC01808191810C94B12095
:102FC000CF93C82F882309F48BC08238C1F40E94A4
:102FD000161681FD85C089E30E94DF200E945321DF
:102FE0002FEF81EE94E0215080409040E1F700C047
:102FF000000089E30E94E620CF910C94532183388E
:10300000A1F40E94161680FD6BC083E50E94DF20AC
:103010000E9453212FEF81EE94E021508040904098
:10302000E1F700C0000083E5E5CF8438A1F40E94F9
:10303000161682FD55C087E40E94DF200E945321AE
:103040002FEF81EE94E0215080409040E1F700C0E6
:10305000000087E4CFCF8CEF8C0F813A90F46C2F77
:1030600080911E0190911F010E94A722882329F0C0
:103070008C2F0E94E6200E9453218C2F0E94DF207B
:10308000BBCF80E28C0F883048F4C77081E001C06C
:10309000880FCA95EAF70E940721AECFEBE5EC0F47
:1030A000E33040F4F0E0E755FE4F808190E0CF91AF
:1030B0000C948B16E8E5EC0FE73150F4F0E0EE0FDE
:1030C000FF1FE558FE4F80819181CF910C94A1168E
:1030D000C03F30F08C2F0E942125CF910C940C26FC
:1030E000CF910895882309F452C0823871F40E9468
:1030F000161681FF4CC089E30E94DF200E945321F5
:1031000089E30E94E6200C945321833859F40E94ED
:10311000161680FF3CC083E50E94DF200E945321E9
:1031200083E5EFCF843859F40E94161682FF2FC032
:1031300087E40E94DF200E94532187E4E2CF9CEFC6
:10314000980F913AF0F290E2980F983050F487700F
:1031500091E001C0990F8A95EAF7892F0E940D210D
:10316000D2CF9BE5980F933020F490E080E00C9450
:103170008B1698E5980F973120F490E080E00C943E
:10318000A116803F20F00E9489250C940C260895FA
:10319000CF93C82F0E94E017C93349F42FEF87EE71
:1031A00093E0215080409040E1F700C000008C2F58
:1031B000CF910C947218882321F00E9407210C945F
:1031C00053210895882321F00E940D210C9453214E
:1031D0000895BF92CF92DF92EF92FF920F931F93C9
:1031E000CF93DF936C01D62FC72FFC010581029589
:1031F0000F70128111110E9427210E94FD20E82EDC
:10320000882391F01123D1F08C2F807F803421F01E
:1032100080E28D0F883090F082E00E949E210E9413
:10322000FD2091E0E82EE926BC2EB2949FE0B92261
:10323000EB2DF0E0E15DFF4C0C94A82FE12CF4CFD6
:103240000C2F0F70C07F11F00295007F1123A9F0A1
:10325000002359F080E28D0F883010F0D11109C0A1
:10326000802F0E9407210E9453218D2F0E94E0177A
:1032700014C0802F0E941A21F6CF8D2F0E94721841
:10328000002359F080E28D0F883010F0D1112CC04E
:10329000802F0E940D210E9453212B2D2850330B8B
:1032A0002430310520F40E9416160E948807EE2073
:1032B00009F49EC10E94F92080FD9AC1F601128294
:1032C0000E94F3200E94801FC6010E94191B0E94C9
:1032D000F320DF91CF911F910F91FF90EF90DF903E
:1032E000CF90BF900C94A11F802F0E942021D3CF9C
:1032F000FC2FFF70FF2EC07FC03219F0F29480EFD8
:10330000F822DD2369F0D13049F1112391F1002336
:1033100051F1F601858180FFA8CF8F70858323C08E
:10332000112381F0011106C00E943A218F290E94C9
:10333000DB18B3CF0130C1F70E943A218F290E94D8
:103340004021ABCF011106C00E9449218F2D0E9460
:10335000E218A3CF013009F4A0CFF6CF112329F052
:10336000063008F09ACF8F2DE2CF053008F095CFC8
:10337000EDCF002359F3D93349F4FFEF27EE33E0C3
:10338000F15020403040E1F700C000008D2F0E9436
:10339000721883CF8C2F86958695837069F0813063
:1033A00009F07BCF8D2F9C2F9370111102C090E0FC
:1033B00080E00E94A11671CF8D2F9C2F9370111168
:1033C00002C090E080E00E948B1667CF8D2F112302
:1033D00029F00E9421250E940C265FCF0E9489259A
:1033E000FACF8C2F837009F041C0111156CF4D2FA9
:1033F000429546954770440F440F0D2F0F7010E013
:1034000030E020E0042E04C0000F111F221F331FE4
:103410000A94D2F760E070E0CB01D4FF0FC06FE0F8
:1034200070E080E090E004C0660F771F881F991F4E
:103430004A95D2F76095709580959095C695C695FA
:10344000C370602B712B822B932BC23049F058F440
:10345000C13019F00E94141F20CF0E94021F1DCFFF
:103460000E94261F1ACF0E94001F17CF8695112396
:1034700011F08C2F8170882309F40FCF4D2F4295C6
:1034800046954770440F440F0D2F0F7010E030E049
:1034900020E0042E04C0000F111F221F331F0A94C6
:1034A000D2F760E070E0CB01D4FF0FC06FE070E0B6
:1034B00080E090E004C0660F771F881F991F4A952F
:1034C000D2F76095709580959095C695C695C37016
:1034D000602B712B822B932BC23049F058F4C130F2
:1034E00019F00E94F71FD9CE0E94E51FD6CE0E9488
:1034F0000920D3CE0E943A1FD0CECF70112329F0DD
:103500008C2F0E94801F8D2F12CF8D2F0E94E218CA
:103510008C2F0E94A11FC1CED23F89F160F4D03F11
:10352000C9F0D13F29F1112309F442C001119DCE08
:103530008C2F8F7121C0D33F39F1D43FA1F71123D4
:1035400069F1CF718C2F0E94801F63E08C2F0E9445
:103550008921A3CE112341F0053008F09ECE8C2F97
:103560008F710E94C41F99CE063008F096CEF7CF17
:103570008C2F8F71112369F20E94801F8ECE8C2FA9
:103580008F711123C9F3C5CF112329F08C2F8F71AF
:103590000E946B1F82CE0E94461F7FCE81E00E9458
:1035A0009E21023008F479CE82E00E949E2175CEE1
:1035B000002359F0D93309F0E9CE8FEF97EEE3E01D
:1035C00081509040E040E1F7DFCE8C2F8F71A1CF8A
:1035D0004C2F4F706D2FC6010E9408080E94781E64
:1035E0005CCE4C2F4F706D2FC6010E940B0855CE3C
:1035F000DF91CF911F910F91FF90EF90DF90CF90CF
:10360000BF9008950F931F93CF93DF93EC016881D0
:1036100079818A810E94BB208C010E941B200E941C
:10362000FF1EB801CE01DF91CF911F910F910C9435
:10363000E918CF93DF93EC018B819C81892B29F0D2
:103640008881998189238F3F59F4DF91CF91089523
:10365000CE010E94021BCE01DF91CF910C9468072E
:10366000CE010E94A0078111F3CF0E94FD20882384
:1036700061F38A81882349F382E0DF91CF910C9432
:103680009E21882321F00E941A210C945321089531
:10369000882321F00E9420210C94532108950E9438
:1036A00027210E9437210E9453210E94B5270E94A2
:1036B0000C2690E080E00E948B1690E080E00C9455
:1036C000A1160E94ED200C944F1B0E9414210C9413
:1036D000611BE92FE295EF70E250EE3070F4F0E0FC
:1036E000E15CFF4C0C94A82F803F19F020F4883E39
:1036F00020F481E00895843FE1F380E00895883E5E
:10370000C0F3813FD1F7F5CF93FB882780F9089567
:103710000E94B1200C94691BCF93DF9300D000D09E
:103720000F92CDB7DEB70F900F900F900F900F90C4
:10373000DF91CF910895CF93DF9300D000D000D0D8
:10374000CDB7DEB726960FB6F894DEBF0FBECDBF5D
:10375000DF91CF9108951F93CF93DF93C091E00144
:1037600016E08091E1018C1304C0DF91CF911F918D
:103770000895D0E01C9FF0011D9FF00D1124EE5123
:10378000FE4F4081518162817381848195810E94C5
:103790009B1B2196C770E5CF4091120250911302F6
:1037A0006091140270911502809116029091170297
:1037B0000C949B1B1F93CF93DF9380911702807F04
:1037C000A9F480911402882389F08091E001C091CE
:1037D000E1016091120270911302A0911502B09163
:1037E0001602D62FD72316E0C81304C0DF91CF915D
:1037F0001F91089590E0109711F0DF3F19F40196A2
:103800008770F2CF189F9001199F300D1124F90194
:10381000EE51FE4F41814713F2CF40814613EFCF67
:1038200042814111ECCF438154814A1B5B0B483CE0
:10383000510528F7809117028F70806180931702DD
:10384000F901E951FE4F80818F708061808382E1B0
:1038500092E00E94191BDF91CF911F910C94AB1B3A
:10386000AF92BF92CF92DF92EF92FF920F931F938E
:10387000CF93DF93CDB7DEB761970FB6F894DEBF75
:103880000FBECDBF8C0185E0F801DE011D960190D1
:103890000D928A95E1F7F80140815181E28082E141
:1038A000C82E82E0D82E6091150270911602611523
:1038B000710509F461C19091120220911302892FC0
:1038C00082238F3F09F458C1A380B480F090140282
:1038D000F501E61BF70BFF2009F4FCC080911702ED
:1038E000382F307FE83CF10508F0B2C0311179C0C3
:1038F000FE2C251323C0941321C0E1101FC08F702C
:103900008061809317020E94CC1BC6010E94191B84
:1039100080911702F80185838F2D61960FB6F89478
:10392000DEBF0FBECDBFDF91CF911F910F91FF90F2
:10393000EF90DF90CF90BF90AF900895AB2829F023
:10394000842F85238F3F09F033C180E0F82FF17079
:10395000DF2E80FF3CC08091E0012091E10136E044
:10396000821315C04D875E878D859E850E94B1208C
:10397000292F22952F702230F0F0243018F59F70F7
:10398000F1F0F8019581907FD1F4D12C1EC090E028
:10399000389FF001399FF00D1124EE51FE4F6181E7
:1039A000651306C06081641303C062816E110FC08D
:1039B00001968770D5CF9F7011F0882331F3805E18
:1039C000883018F3C8010E94191BFD2CA5CFEE20EA
:1039D00009F4A2CF80911702816080931702F12C25
:1039E0009BCF251306C0941304C0F801EE2009F400
:1039F0008DC04D875E878D859E850E94881B88239C
:103A000019F1EE2009F180911702803270F02091B7
:103A100012023091130238872F831986BB86AA863B
:103A20008C87CE0107960E94191B86E0F801A2E15F
:103A3000B2E001900D928A95E1F70E94DA1B0E9494
:103A4000CC1BFF24F39468CFC8010E94191BF9CF47
:103A5000311113C07A2DB98AA88A6E2D89890E94E6
:103A60008C1B82E192E00E94191B86E0F601119204
:103A70008A95E9F70E94CC1BB2CF25130FC094138F
:103A80000DC0E1100BC0F8018583C8010E94191B0D
:103A900086E0F60111928A95E9F73ECF4D875E8761
:103AA0008D859E850E94881B882371F2EE2061F22D
:103AB00080911702803208F4B8CF20911202309121
:103AC00013023A8329831B82BD82AC828E83CE018E
:103AD0000196A9CFE83CF10508F041C0FE2CEE208C
:103AE00009F4B2CF25132AC0941328C0809117027D
:103AF00080FD1BC0982F907FC1F0F8018583903F17
:103B000031F0982F907F905F8F70892B8583C8014B
:103B10000E94191B86E0F801A2E1B2E001900D922B
:103B20008A95E1F70E94CC1BF7CE86E0F801A2E16E
:103B3000B2E001900D928A95E1F7EECE4D875E8757
:103B40008D859E850E94881B81116FCF8091170201
:103B5000816080931702C8010E94191BDDCE7A2D67
:103B6000B98AA88A6E2D89890E948C1B86E0F6018D
:103B700011928A95E9F7D6CFEE2009F465CF4D87EB
:103B80005E878D859E850E94881BF82E882309F408
:103B90005BCF86E0F801A2E1B2E001900D928A9538
:103BA000E1F782E192E00E94DB170E94DA1BBACFB4
:103BB00081E08E25CBCE88EC90E008951F93CF93C3
:103BC000DF93CDB7DEB72C970FB6F894DEBF0FBEEC
:103BD000CDBF4F83588769877A878B879C87CE01B3
:103BE00007960E94301C882369F08A859B85892B63
:103BF00039F04F815885842F85238F3F09F071C09C
:103C000016E05FC086E0FE013796DE011196019056
:103C10000D928A95E1F78A859B85892B89F38F819F
:103C2000988589238F3F61F32091E10130E0C9013C
:103C30000196877099274091E0014817190671F4A1
:103C40000E94651B1092E1011092E00186E0E2E122
:103C5000F2E0DF011D928A95E9F7D2CF96E0929FBC
:103C6000D001939FB00D1124AE51BE4FFE0131968D
:103C700001900D929A95E1F78093E1010E94AB1BB0
:103C8000BFCF819FC00111248E519E4F0E94301CD6
:103C90008823E9F0E091E0011E9FF0011124EE512C
:103CA000FE4F4081518162817381848195810E94A0
:103CB0009B1B8091E00190E001968770992780938B
:103CC000E0018091E0019091E1018913DACF2C9617
:103CD0000FB6F894DEBF0FBECDBFDF91CF911F911D
:103CE000089569857A858B859C850E949B1B88CF6A
:103CF000EF92FF920F931F93CF93DF938C01892B49
:103D000081F0F12CEE24E394E8012196F8018491EE
:103D1000843770F4843008F05FC08130B1F08230B5
:103D2000A1F1DF91CF911F910F91FF90EF90089536
:103D3000853709F44CC008F43DC09CE7980F9037D4
:103D400080F78F770E94721849C00E5F1F4FFE01E7
:103D5000849190E2980F983060F48770FE2D01C036
:103D6000FF0F8A95EAF78F2F0E942A210E94532184
:103D700002C00E94E0178F2D815030F2EFE9FFE082
:103D80003197F1F700C00000F7CF0E5F1F4FFE0123
:103D9000849190E2980F983050F48770FE2D01C006
:103DA000FF0F8A95EAF78F2F0E943021DFCF0E9404
:103DB0007218E1CF0E5F1F4FFE01C491C150D8F2BF
:103DC0008FE99FE00197F1F700C00000F7CF0E5F89
:103DD0001F4FFE01F490CFCF0E94E0178E01CBCF92
:103DE00008950C94F01E0E94F11E60934E02709391
:103DF0004F0280935002909351020C944F1B0895F0
:103E00000C94F31E0F931F9300914E0210914F02DA
:103E10002091500230915102602B712B822B932BF9
:103E20001F910F910C94F31E0F931F9300914E025C
:103E300010914F0220915002309151026023712362
:103E4000822393231F910F910C94F31E0F931F93C2
:103E500000914E0210914F02209150023091510278
:103E600060277127822793271F910F910C94F31ECF
:103E70000C942B060E94381F60934A0270934B02E9
:103E800080934C0290934D020C944F1B60E070E0C5
:103E9000CB010C943A1F611571058105910529F438
:103EA00081E0442361F080E00895DC01CB0104C08F
:103EB000B695A795979587954A95D2F781700895FD
:103EC000482F60914A0270914B0280914C02909170
:103ED0004D020C944B1F0F931F9341E050E060E0A4
:103EE00070E08A019B0104C0000F111F221F331FC5
:103EF0008A95D2F7C901B8011F910F910C943A1F0E
:103F00000F931F9341E050E060E070E004C0440F65
:103F1000551F661F771F8A95D2F780914A029091AC
:103F20004B02A0914C02B0914D028A019B01082BDB
:103F3000192B2A2B3B2BC901B8011F910F910C940F
:103F40003A1F0F931F9341E050E060E070E004C01F
:103F5000440F551F661F771F8A95D2F7CB01BA0110
:103F6000609570958095909500914A0210914B0252
:103F700020914C0230914D026023712382239323C0
:103F80001F910F910C943A1F0F931F9341E050E043
:103F900060E070E004C0440F551F661F771F8A95CC
:103FA000D2F780914A0290914B02A0914C02B091BD
:103FB0004D028A019B01082719272A273B27C9019F
:103FC000B8011F910F910C943A1F0F931F9300910A
:103FD0004A0210914B0220914C0230914D02602B0D
:103FE000712B822B932B1F910F910C943A1F0F93DF
:103FF0001F9300914A0210914B0220914C02309184
:104000004D0260237123822393231F910F910C94FF
:104010003A1F0F931F9300914A0210914B02209177
:104020004C0230914D0260277127822793271F9100
:104030000F910C943A1F08959295907F890F982FB5
:10404000977041E001C0440F9A95EAF786958695EE
:10405000869595E0899FF0011124E85EFD4F30E0E0
:1040600020E070E05191DF011197CB01022E02C0D8
:10407000969587950A94E2F7817081958527842328
:1040800085278C932F5F3F4F2530310559F70895D1
:104090009295907F890F982F977086958695869533
:1040A00025E0829FF0011124E85EFD4F50E040E0E2
:1040B00080E0219130E0092E02C0369527950A94C0
:1040C000E2F721703327042E01C0220F0A94EAF789
:1040D000822B4F5F5F4F4530510559F70895BF92CE
:1040E000CF92DF92EF92FF920F931F93CF93DF93C4
:1040F0008C01C0904A02D0904B02E0904C02F090AC
:104100004D0280914E0290914F02A0915002B091C9
:104110005102C82AD92AEA2AFB2ACFE1D0E0BC2ED4
:10412000D701C6010C2E04C0B695A7959795879523
:104130000A94D2F780FD0EC0219788F7B12C8B2D01
:10414000DF91CF911F910F91FF90EF90DF90CF9073
:10415000BF900895B8018C2F0E942908019761F340
:10416000EECFCF93DF93EC010E946F20BE01DF9171
:10417000CF910C9429081F93CF93DF93EB0190917B
:10418000DF01992331F0CB01DF91CF911F910C9486
:10419000B120882379F0CB010E946F20182F682F5F
:1041A000CE010E941C20BE01812FDF91CF911F9173
:1041B0000C942908CB010E944820182FF4CF682FB7
:1041C00080911E0190911F010C944923682F8091CA
:1041D0001E0190911F010C94542380911E01909117
:1041E0001F010C945F2380915202859585958595DA
:1041F00008958091520287700895909152029770AD
:1042000081E009F480E0089580917602089590910C
:104210007602892B8093760208958095909176029C
:1042200098239093760208951092760208958091D3
:104230007502089590917502892B809375020895F7
:10424000809590917502982390937502089510922D
:104250007502089590917402892B809374020895D9
:10426000809590917402982390937402089510920F
:104270007402089580915302089508950C943D218D
:1042800090915302981721F0809353020C943E2191
:10429000089580915302882329F01092530280E000
:1042A0000C943E210895E0911E01F0911F01809130
:1042B00076028083E0911E01F0911F018081909130
:1042C0007502892B8083E0911E01F0911F0180818E
:1042D00090917402892B808390915302992381F0ED
:1042E000E0911E01F0911F018081892B80838091D4
:1042F0001E0190911F010E94932281110E94492169
:1043000080911E0190911F010C94221608950C9427
:10431000862198E0899F90011124622B60935202BC
:104320000E94801F809152028595859585950C94F9
:1043300087211092520280E00C94872190915202C2
:104340008095892380935202282F277071F4282F9B
:10435000082E000C330B9217130639F085958595BE
:1043600085950E94A11F0C94992108959093BD01F9
:104370008093BC010895829590E09C01220F331F29
:10438000220F331F2C7C9595879595958795837380
:10439000282B30E0C901880F991F8A7A3595279517
:1043A0002575822B0895CF93DF93D92F0E94BB21CF
:1043B000C82F8D2F0E94BB219C2FDF91CF91089594
:1043C0006FEF7FEF90E080E00C94033090E080E0AE
:1043D0000E94DF2F21E08C3E9E4F09F020E0822FCB
:1043E000089582E090E00C94D12F83E090E00C944B
:1043F000D12FCF9384E090E00E94D12FC82F81E28B
:1044000090E00E94D12F982F8C2FCF910895CF93B9
:10441000C92F682F84E090E00E94E52F6C2F81E285
:1044200090E0CF910C94E52F86E090E00C94D12F92
:10443000682F86E090E00C94E52FAB01BC018FE083
:1044400090E00C94F72FAB01BC0183E190E00C9459
:10445000F72F60E070E0CB010C94232260E070E065
:10446000CB010E941D220C9429226CEE7EEF90E07D
:1044700080E00E94033060E082E090E00E94E52F3F
:1044800060E083E090E00E94E52F10924E021092CF
:104490004F02109250021092510260E084E090E0CE
:1044A0000E94E52F60E081E290E00E94E52F60E04D
:1044B00085E090E00E94E52F60E086E090E00E94B9
:1044C000E52F6FEF87E090E00E94E52F40E050E09D
:1044D000BA0188E090E00E94F72F60E08DE090E064
:1044E0000E94E52F40E050E0BA0188E190E00E9490
:1044F000F72F60E087E190E00E94E52F40E050E078
:10450000BA018CE190E00E94F72F60E080E290E039
:104510000E94E52F0C942E220C943522682F8EE0F9
:1045200090E00C94E52FFC013296809132018823B3
:1045300021F08091AD029EE187FF96E080E09150EE
:1045400008F4089521912223D1F38F5FF8CF6623D9
:1045500001F1209132012223F1F02091AD0227FFD9
:104560001AC0462F4695469546954E3190F4677091
:1045700021E030E002C0220F331F6A95E2F7840F7A
:10458000911DFC01828190E02823392381E0232BB7
:1045900069F480E00895FC0132960896219126176F
:1045A00021F0E817F907D1F7F4CF81E008959C01D5
:1045B000FC0132969FEF80E04191461751F09F3FFA
:1045C00019F4411101C0982F8F5F8630A9F79F3FE2
:1045D00009F40895290F311D97FD3A95F901628379
:1045E0000895FC01329608962191261303C0DF013D
:1045F00011971C92E817F907B9F70895E62FE69589
:10460000E695E695EE3170F4E80FF92FF11D67702D
:1046100021E030E001C0220F6A95EAF78281822B07
:10462000828308958091770280FF0CC01F926F9360
:1046300085EC97E09F938F930E94F6050F900F9063
:104640000F900F900895E62FE695E695E695EE31EA
:1046500078F4E80FF92FF11D677021E030E001C018
:10466000220F6A95EAF720958281282322830895F4
:104670008091770280FF0CC01F926F9387EA97E0CA
:104680009F938F930E94F6050F900F900F900F90BD
:10469000089520913201222329F02091AD0227FDB7
:1046A0000C94FE220C94D72220913201222329F06F
:1046B0002091AD0227FD0C9423230C94F122FC01E0
:1046C000329680913201882351F08091AD0287FFAC
:1046D00006C08EE1DF011D928A95E9F7089586E014
:1046E000F9CF089508950C9472230E94732380914A
:1046F0000D03843009F43AC01092780288E190E00A
:1047000020E40FB6F894A895809360000FBE209324
:10471000600080E00E94F01180E00E948807809194
:10472000790281110AC081E0809379028091C302ED
:10473000817080937A020E94060E0E94732383B7D1
:10474000817F846083BF83B7816083BF78948895BD
:1047500083B78E7F83BF0FB6F894A89580916000D1
:10476000886180936000109260000FBE08950895E4
:10477000CF930E9471230E94D60A0E94B723C0E003
:104780008C2F0E941A0A892B31F4CF5FC530C1F7F4
:1047900080E0CF91089581E0FCCF08950C94CD2363
:1047A0000E94651B0E9486100E9416160E948807B0
:1047B0001092790280917A0281110E94F10F0C947B
:1047C000CE231F921FB61F9211248F939F93AF93F6
:1047D000BF9380917802811113C08091050390915D
:1047E0000603A0910703B09108034196A11DB11DD6
:1047F0008093050390930603A0930703B0930803E7
:10480000BF91AF919F918F911F901FBE1F901895E0
:1048100082E084BD93E095BD9AEF97BD80936E00D2
:1048200008952FB7F8948091050390910603A09105
:104830000703B09108032FBF08959C014FB7F89468
:104840008091050390910603A0910703B09108039E
:104850004FBF821B930B089578941F921FB61F922F
:1048600011248F939F93AF93BF93809105039091F1
:104870000603A0910703B09108030196A11DB11D85
:104880008093050390930603A0930703B093080356
:10489000BF91AF919F918F911F901FBE1F90189550
:1048A00081E08093E00080E28093D8001092C900FC
:1048B0008FE19EE40197F1F700C0000087E090EBE4
:1048C000DC018093160390931703A0931803B09311
:1048D000190388E19CE00FB6F894A89580936000D6
:1048E0000FBE90936000FFCF0C94E0210E94D60A87
:1048F0008FE39CE90197F1F700C000000E94D60AFF
:1049000080E00E941A0A80FF04C00E9474240C9464
:10491000502408950E94E621811102C00E948C2239
:104920000E94F121809377020E94F9219093AE02B8
:104930008093AD020E94F521682F70E090E080E046
:104940000E94001F60914A0270914B0280914C02BC
:1049500090914D020C94381F8091810280FD32C0ED
:1049600081FF10C06091250185E0689FB00111248E
:10497000759567956038710570F56115710569F178
:10498000862F089582FD21C080918002882301F145
:104990009091240160912501891728F085E0689F96
:1049A000B0011124E7CF869FB001112485E0869FD6
:1049B0009001879F300D1124692F70E0C9010E947A
:1049C000722FD8CF61E070E0DBCF6FE770E0D8CF17
:1049D00065E070E0D5CF8FE7089581E0089580917C
:1049E000810280FD29C081FF0AC06091210170E031
:1049F000759567956115710511F1862F089582FDF2
:104A000018C0909180029923B9F0609120018091A3
:104A10002101961738F0682F70E06038710550F367
:104A20008FE70895899FC001112470E00E94722FC2
:104A3000F4CF6FE770E0E1CF61E070E0DECF81E0BE
:104A40000895803F31F40E94AC24819580938502C3
:104A50000895813F19F40E94AC24F8CF823F31F4CD
:104A60000E94AC248195809384020895833F19F4B9
:104A70000E94AC24F8CF893F29F40E94EF24809350
:104A8000860208958A3F21F40E94EF248195F7CF92
:104A90008B3F31F40E94EF24819580938702089523
:104AA0008C3F19F40E94EF24F8CF843F31F48091B9
:104AB00083028160809383020895853F21F4809171
:104AC00083028260F7CF863F21F480918302846065
:104AD000F1CF873F21F4809183028860EBCF883F3C
:104AE00021F4809183028061E5CF8D3F31F4809184
:104AF000810281608093810208958E3F21F480912C
:104B000081028260F7CF8F3FB9F780918102846084
:104B1000F1CF90918402803F59F48091850287FF04
:104B20000DC01092850291110BC01092800208C036
:104B3000813F81F48091850218169CF3992381F0BE
:104B40008091860290918702892B09F064C01092AF
:104B50007F020895823F49F497FFF0CF10928402BC
:104B6000809185028111ECCFE0CF833F19F41916B3
:104B7000ACF3E4CF20918602893F29F41216F4F6B3
:104B800010928602DBCF8A3F19F427FFD7CFF8CFE8
:104B9000209187028B3F29F427FFD0CF1092870204
:104BA000CDCF8C3F19F41216CCF3C8CF843F31F42B
:104BB000809183028E7F80938302C0CF853F21F452
:104BC000809183028D7FF7CF863F21F4809183020D
:104BD0008B7FF1CF873F21F480918302877FEBCFDA
:104BE000883F21F4809183028F7EE5CF8D3F31F4A1
:104BF000809181028E7F80938102A0CF8E3F21F42D
:104C0000809181028D7FF7CF8F3F09F097CF809100
:104C100081028B7FF0CF08958091770283FF7EC061
:104C20008AE098E00E945D05809183021F928F9335
:104C300085E098E09F938F930E94F60583E098E0CB
:104C40000E945D0580918402282F082E000C330BF2
:104C50003F938F9380E098E09F938F930E94F60597
:104C60008EEF97E00E945D0580918502282F082E27
:104C7000000C330B3F938F938BEF97E09F938F93B1
:104C80000E94F60589EF97E00E945D0580918602FB
:104C9000282F082E000C330B3F938F9386EF97E05D
:104CA0009F938F930E94F60584EF97E00E945D0525
:104CB00080918702282F082E000C330B3F938F938F
:104CC00081EF97E09F938F930E94F6058EEE97E019
:104CD0000E945D05809180021F928F938BEE97E07A
:104CE0009F938F930E94F60589EE97E00E945D05E1
:104CF000809181021F928F9386EE97E09F938F930E
:104D00000E94F60583EE97E00E945D058DB79EB781
:104D10004C960FB6F8949EBF0FBE8DBF0E94112413
:104D20009C019091840280918502982B21F0309310
:104D30007E0220937D029091860280918702982BBB
:104D400021F030937C0220937B0282E892E00C9465
:104D50007D16EF92FF920F931F93CF93DF9300D0B6
:104D600000D000D0CDB7DEB786E0E2E8F2E0DE01A9
:104D7000119601900D928A95E1F7E0908402F090EF
:104D8000850200918602109187021092840210928F
:104D9000850210928602109287028E2D8F2991F043
:104DA00080917D0290917E020E941D24AC01909121
:104DB0008002992309F43FC08091260184171506CB
:104DC00008F447C0802F812B91F080917B02909155
:104DD0007C020E941D24AC0190917F02992309F46A
:104DE00077C0809122018417150608F47FC0809156
:104DF000840290918502892B90918602892B909153
:104E00008702892B11F00E940C2686E0FE01319664
:104E1000A2E8B2E001900D928A95E1F726960FB6CE
:104E2000F894DEBF0FBECDBFDF91CF911F910F91E0
:104E3000FF90EF900895209127018AE0289F90012C
:104E400011242417350708F0BDCF9F5F909380028F
:104E500002C09F3FD1F7EE2059F00E94AC249FEF93
:104E60001E140CF491E0899F802D112480938402FC
:104E7000FF2059F00E94AC249FEF1F140CF491E026
:104E8000899F802D112480938502309184023323E1
:104E900009F498CF20918502222309F493CF45EBA2
:104EA0003403C0011124992359F09093840245EBF7
:104EB000240390011124332339F03093850282CFEB
:104EC00081E080938402F3CF81E0809385027ACFE2
:104ED000209123018AE0289F90011124241735078F
:104EE00008F085CF9F5F90937F0202C09F3FD1F76C
:104EF000002359F00E94EF249FEF10160CF491E06C
:104F0000899F802D112480938602112359F00E94DD
:104F1000EF249FEF11160CF491E0899F802D11244E
:104F20008093870230918602332309F460CF209169
:104F30008702222309F45BCF45EB3403C00111241F
:104F4000992359F09093860245EB24039001112494
:104F5000332339F0309387024ACF81E08093860271
:104F6000F3CF81E08093870242CF86E0E2E8F2E06F
:104F7000DF011D928A95E9F71092800210927F025C
:104F80001092810208958091AB0208959FB7F89422
:104F900010928A029FBF90910D03943009F048C08F
:104FA0002091E9002F703091EC00932F917030FD2B
:104FB00090E8922B23E02093E9002091EB0020FF62
:104FC00034C02091EE0027FF30C0209188022223B8
:104FD00021F02091E80025FF28C01092880226E0E9
:104FE0003091E80035FF14C08093F1008091E80013
:104FF00085FD27C08091E80080FFFCCF8091E8000C
:105000008E778093E8009F709093E90080E0089588
:1050100030910D03343049F43091EB0035FD05C07B
:10502000215041F481E0809388029F709093E900C1
:105030008FEF0895EFE9FFE03197F1F700C000002E
:10504000CFCF8FB7F89421E020938A028FBFDBCFB8
:10505000CF93DF9300D00F92CDB7DEB790910D03C1
:10506000943019F589837B836A8382E08093E90019
:105070008FEF9091E800815095FD06C095ED9A95CF
:10508000F1F700008111F5CF8091E80085FF0DC098
:1050900050E040E063E070E0CE0101960E94B22A49
:1050A0008091E8008E778093E8000F900F900F902A
:1050B000DF91CF910895BC0184E00C942828BC01B5
:1050C00083E00C9428289C0182E08093E9009FEF04
:1050D0008091E800915085FD06C085ED8A95F1F735
:1050E00000009111F5CF8091E80085FF0CC050E0E1
:1050F00040E066E070E0C9010E94B22A8091E800B9
:105100008E778093E8000895CF93DF93EC01809130
:1051100032018823B1F18091AD0287FF32C060E295
:1051200082E08093E9008FEF9091E800815095FD37
:1051300006C095ED9A95F1F700008111F5CF8091A9
:10514000E80085FF1BC08091320170E050E040E034
:10515000811104C050E040E068E070E0CE010E94A0
:10516000B22A8091E8008E778093E80080E2FE0109
:10517000ABE8B2E001900D928A95E1F7DF91CF9113
:10518000089568E081E0CDCF82E598E00E945D055A
:1051900080910C03811109C00E94422C0E949F2C17
:1051A0008091E20084608093E20008958EE498E0AC
:1051B0000E945D0510920C0308958AE498E00C9417
:1051C0005D0586E498E00C945D0582E498E00E9419
:1051D0005D050C94D023209189022F5F822F62E31A
:1051E0000E94522F992319F020938902089510925A
:1051F000890280918A028823F1F080910D03843026
:10520000C1F49091E9009F702091EC00822F817091
:1052100020FD80E8892B93E09093E9009091EB00CA
:1052200090FF04C09091EE0097FD08C08F708093AE
:10523000E90010928A0208951092F1009091E8001E
:1052400095FDFACF9091E80090FFF0CF9091E800A3
:105250009E779093E800EACF42E061EC81E00E9403
:10526000BE2B42E261EC82E00E94BE2B42E261EC86
:1052700083E00C94BE2B80910F03833009F45FC050
:1052800030F48130C1F1823009F49BC008958A3036
:1052900009F487C08B3009F46DC0893009F04EC025
:1052A00080910E03813209F049C0809112039091E0
:1052B0001303029708F042C08091E800877F809333
:1052C000E8008091E80082FF35C09091F300809162
:1052D000F200029729F48091F1008B7F813021F454
:1052E0008091F1008093AB028091E8008B778093EE
:1052F000E8000C94F22B80910E03813AF9F480912E
:10530000E800877F8093E800809112039091130357
:10531000892B61F460E28BE892E070E00E94012B3F
:105320008091E8008B778093E800089560E090E03A
:1053300080E0F3CF80910D038111C3CF0895809158
:105340000E03813AD9F78091120390911303892BB0
:10535000A9F78091E800877F8093E8008091E800BA
:1053600080FFFCCF809132018093F1008091E800B2
:105370008E77BDCF80910E03813201F780911203A9
:1053800090911303892BD1F68091E800877F809359
:10539000E8000E94F22B80911003809332010C945C
:1053A000651B80910E03813249F68091E800877F6A
:1053B0008093E8000E94F22B809111038093AC024D
:1053C000089580910E03813A09F0B8CF8091E800EA
:1053D000877F8093E8008091E80080FFFCCF809178
:1053E000AC02C2CF84B7877F84BF0FB6F894A8956C
:1053F00080916000886180936000109260000FBE11
:1054000080E890E00FB6F89480936100909361007B
:105410000FBE0E94C4160E94422C0E949F2C8091B5
:10542000E20084608093E20086EC97E20E94B6215D
:1054300078940E94272F0E94CE1688E291E00E9465
:10544000111681E398E00E945D0580910D0385307F
:1054500019F00E940217F9CF8DE298E00E945D05D5
:105460000E94752380910B03882379F30E94B8234F
:10547000882359F30E949C2AE8CF0C943F2A292FB5
:1054800033272330310521F168F42130310509F447
:1054900049C02230310509F44AC090E080E030E094
:1054A00020E029C02132310581F122323105A9F7EE
:1054B0006330710590F7FB01EE0FFF1FE155FE4FC2
:1054C0002081318164557E4FFB01808190E013C0C3
:1054D00099278130910599F0009741F0823091052C
:1054E00089F00397D1F6E6E5F8E002C0E0E8F8E0DD
:1054F000849190E09F01FA01318320830895EEE6C4
:10550000F8E0F6CFECE5F8E0F3CF6330710528F66C
:10551000660F771FFB01EB54FE4F2081318189E03C
:1055200090E0E9CF82E190E02FED38E0E4CF8BE529
:1055300090E024E838E0DFCF80E189BD82E189BDD9
:1055400009B400FEFDCF8091D8008F7D8093D800F4
:105550008091E00082608093E0008091E00081FD16
:10556000FCCF0895AF92BF92CF92DF92FF920F933C
:105570001F93CF93DF936C01EB018A010E94112CE2
:10558000F82E811123C00115110539F0F801808131
:105590009181C81BD90BC80ED91EB12CA12C209704
:1055A000A9F08091E80085FD22C08091E8008E7707
:1055B0008093E80001151105A1F0F8018081918127
:1055C000A80EB91EB182A08285E0F82E8F2DDF9142
:1055D000CF911F910F91FF90DF90CF90BF90AF9030
:1055E00008950E94112C8823D1F2F82EEFCFF601F6
:1055F00081916F018093F1002197FFEFAF1ABF0AED
:10560000CECFFC0180911403909115038617970764
:10561000A0F06115710529F49091E8009E779093B0
:10562000E80090E06115710551F4911108C0809176
:10563000E80082FF34C080E00895BC01F2CF809181
:105640000D038823C1F18530C1F18091E80083FD0D
:1056500030C08091E80082FDEACF8091E80080FFB1
:10566000E1CF8091F3002091F200382F6115710590
:1056700019F02830310558F091E02830310509F053
:1056800090E02091E8002E772093E800CBCF819125
:105690008093F100615071092F5F3F4FE7CF8091F8
:1056A0000D03882341F0853041F08091E80083FFAD
:1056B000BECF81E0089582E0089583E00895FC0163
:1056C000809114039091150386179707A0F0611538
:1056D000710529F48091E8008E778093E80090E0CE
:1056E0006115710551F4911108C08091E80082FFA5
:1056F00035C080E00895BC01F2CF80910D0388236E
:10570000C9F18530C9F18091E80083FD31C08091F5
:10571000E80082FDEACF8091E80080FFE1CF809130
:10572000F3002091F200382F6115710519F028302F
:10573000310558F091E02830310509F090E0809172
:10574000E8008E778093E800CBCF84918093F100BE
:105750003196615071092F5F3F4FE6CF80910D0365
:10576000882341F0853041F08091E80083FFBDCF70
:1057700081E0089582E0089583E00895982F97309E
:1057800028F08F708093E90081E008959093E900FC
:10579000242F762F50E0981731F07091EC00209173
:1057A000ED005091F00021FD02C09F5FE8CF3091E5
:1057B000EB003E7F3093EB003091ED003D7F309366
:1057C000ED003091EB0031603093EB007093EC0012
:1057D0002093ED005093F0002091EE0027FDE5CFDF
:1057E00080E0089580910E0387FF13C08091E80048
:1057F00082FF06C08091E8008B778093E80004C0A8
:1058000080910D038111F2CF089580910D038823BB
:10581000D9F38091E80080FFF8CF8091E8008E777F
:10582000ECCF2091E4003091E50095E6A9012091AC
:10583000EC00822F817020FF06C08091E80080FF7D
:1058400006C080E008952091E80022FD1AC08091F2
:105850000D03882389F0853089F08091EB0085FD68
:105860000FC02091E4003091E50042175307F9F290
:105870009150E1F684E0089582E0089583E0089570
:1058800081E008950E94B02C0E94B82CE0EEF0E078
:10589000808181608083E8EDF0E080818F77808374
:1058A00019BCA7EDB0E08C918E7F8C9380818F7EA8
:1058B000808310920C0308950F931F93CF93DF936F
:1058C0000E94B02C0E94B82CC8EDD0E088818F7760
:1058D000888388818068888388818F7D888319BCCC
:1058E00010920D031092090310920B0310920A03F9
:1058F00000EE10E0F80180818B7F808388818160D9
:10590000888342E060E080E00E94BE2BE1EEF0E0A0
:1059100080818E7F8083E2EEF0E0808181608083F1
:10592000808188608083F80180818E7F8083888178
:1059300080618883DF91CF911F910F910895E8EDE9
:10594000F0E080818F7E8083E7EDF0E080818160F0
:10595000808384E082BF81E080930C030C945C2CF4
:10596000E8EDF0E080818E7F80831092E200089560
:105970001092DA001092E10008951F920F920FB674
:105980000F9211242F933F934F935F936F937F93C5
:105990008F939F93AF93BF93EF93FF938091E10019
:1059A00082FF0BC08091E20082FF07C08091E1007E
:1059B0008B7F8093E1000E94EB288091DA0080FFCA
:1059C00019C08091D80080FF15C08091DA008E7FC9
:1059D0008093DA008091D90080FF96C080E189BD74
:1059E00082E189BD09B400FEFDCF81E080930D0303
:1059F0000E94C4288091E10080FF19C08091E200DC
:105A000080FF15C08091E2008E7F8093E20080913C
:105A1000E20080618093E2008091D80080628093F0
:105A2000D80019BC85E080930D030E94E128809185
:105A3000E10084FF2BC08091E20084FF27C080E159
:105A400089BD82E189BD89B5982F917080FFFBCF18
:105A50008091D8008F7D8093D8008091E1008F7E67
:105A60008093E1008091E2008F7E8093E20080913C
:105A7000E20081608093E20080910903882309F4A9
:105A800049C084E080930D030E94E5288091E100E5
:105A900083FF29C08091E20083FF25C08091E1004F
:105AA000877F8093E10082E080930D0310920903C9
:105AB0008091E1008E7F8093E1008091E2008E7FF3
:105AC0008093E2008091E20080618093E20042E0F6
:105AD00060E080E00E94BE2B8091F000886080939F
:105AE000F0000E94DD28FF91EF91BF91AF919F914F
:105AF0008F917F916F915F914F913F912F910F9077
:105B00000FBE0F901F90189519BC10920D030E94A4
:105B1000D62870CF8091E30087FD93E090930D032A
:105B2000B3CF1F920F920FB60F9211242F933F9372
:105B30004F935F936F937F938F939F93AF93BF9395
:105B4000CF93DF93EF93FF93D091E900DF708091C3
:105B5000EC00C82FC17080FDC0E81092E900809170
:105B6000F000877F8093F00078940E94D52D1092EA
:105B7000E9008091F00088608093F000CD2BCF7019
:105B8000C093E900FF91EF91DF91CF91BF91AF9169
:105B90009F918F917F916F915F914F913F912F9145
:105BA0000F900FBE0F901F9018951F93CF93DF9308
:105BB000CDB7DEB7AA970FB6F894DEBF0FBECDBF44
:105BC0008EE093E02091F100FC012193CF01F3E0FE
:105BD00086319F07B9F70E943B298091E80083FF37
:105BE0001EC180910E0390910F039A3008F017C1E7
:105BF000E92FF0E0E35BFF4C0C94A82F803899F07C
:105C0000823809F00CC1809112038F70873008F040
:105C100006C18093E9008091EB0085FB882780F91D
:105C20001092E90006C080910A0390910B03911134
:105C300082609091E800977F9093E8008093F10054
:105C40001092F1008091E8008E77E5C0882309F476
:105C5000D3C0823009F0E3C0809110038111D6C017
:105C6000809112038F702FEF280F263008F0D7C0D5
:105C70008093E9002091EB0020FFC8C0933031F4FD
:105C80008091EB0080628093EB00C0C09091EB00AC
:105C900090619093EB0021E030E001C0220F8A95E3
:105CA000EAF72093EA001092EA008091EB00886006
:105CB000EACF8111B4C0109110031F778091E300E7
:105CC0008078812B8093E3008091E800877F809328
:105CD000E8000E94F22B8091E80080FFFCCF8091C9
:105CE000E30080688093E30082E0111183E08093F9
:105CF0000D0395C08058823008F091C08091100348
:105D0000909111038C3D23E09207A1F583E08A83F3
:105D10008AE289834FB7F894DE01139620E03EE0D3
:105D200051E2E32FF0E050935700E49120FF03C0CD
:105D3000E295EF703F5FEF708E2F90E0EA30C0F099
:105D4000C7968D939D932F5F243159F74FBF809154
:105D5000E800877F8093E8006AE270E0CE01019658
:105D60000E94012B8091E8008B778093E80057C058
:105D7000C096E7CF6091120370911303AE014F5F9D
:105D80005F4F0E943D2ABC01892B09F448C09091C5
:105D9000E800977F9093E80089819A810E945F2BA9
:105DA000E1CF8038E1F58091E800877F8093E800BB
:105DB000809109038093F10045CF811130C090910B
:105DC0001003923060F58091E800877F8093E800AF
:105DD000909309030E94F22B80910903882311F00C
:105DE00084E005C08091E30087FDFACF81E08093D5
:105DF0000D030E942C2913C080911003813079F487
:105E000081E0933009F080E080930B031092E90069
:105E10008091E800877F8093E8000E94F22B8091B8
:105E2000E80083FF0AC08091E800877F8093E80044
:105E30008091EB0080628093EB00AA960FB6F894F5
:105E4000DEBF0FBECDBFDF91CF911F910895CF93DD
:105E500080910D038823A1F0C091E900CF7090914B
:105E6000EC00892F817090FD80E8C82B1092E9002A
:105E70008091E80083FD0E94D52DCF70C093E9008A
:105E8000CF910895DB018F939F930E94BD2FBF9107
:105E9000AF91A29F800D911DA39F900DB29F900D79
:105EA00011240895991B79E004C0991F961708F0F2
:105EB000961B881F7A95C9F780950895AA1BBB1B6E
:105EC00051E107C0AA1FBB1FA617B70710F0A61BFA
:105ED000B70B881F991F5A95A9F780959095BC011B
:105EE000CD01089597FB072E16F4009407D077FD97
:105EF00009D00E945E2F07FC05D03EF49095819555
:105F00009F4F0895709561957F4F0895A1E21A2ED5
:105F1000AA1BBB1BFD010DC0AA1FBB1FEE1FFF1F4D
:105F2000A217B307E407F50720F0A21BB30BE40B9D
:105F3000F50B661F771F881F991F1A9469F76095E4
:105F40007095809590959B01AC01BD01CF0108959E
:105F5000EE0FFF1F0590F491E02D0994A29FB00170
:105F6000B39FC001A39F700D811D1124911DB29F8D
:105F7000700D811D1124911D08950E94AE2FA59FC3
:105F8000900DB49F900DA49F800D911D1124089534
:105F9000FB01DC0102C005900D9241505040D8F742
:105FA0000895F999FECF92BD81BDF89A992780B5E1
:105FB0000895A6E1B0E044E050E00C940B30A8E175
:105FC000B0E042E050E00C940B30262FF999FECF60
:105FD00092BD81BDF89A019700B4021639F01FBA3C
:105FE00020BD0FB6F894FA9AF99A0FBE0895039659
:105FF000272F0E94E62F0E94E52F252F0E94E62FD3
:10600000242F0C94E62F0196272F0E94E62F0C9444
:10601000E52FDC01CB01FC01F999FECF06C0F2BDF2
:10602000E1BDF89A319600B40D9241505040B8F756
:106030000895F894FFCF44104C10531058105D1081
:10604000621067106C10711076107B108010461073
:1060500046104610461046104610461046102019AD
:10606000201978197819CA19E6194D194D19F1191D
:106070007D1A8C1A8C1AE81A4D194D19F11A741BD5
:10608000741B7D1B7D1B7F1B7D1B7D1B7D1B741B60
:10609000741B841B7D1B7D1B841BFE2D262E0F2F46
:0E60A000262E0F2F592E7A2E0F2FD12EDD2EE9
:1060AE0001000000AB060F0600000000000000001B
:1060BE0000000000000000000014001414FF540241
:1060CE00140A32110F051411C327842863285F2880
:1060DE005B2801E200E900EA00B500B600B700CD8A
:1060EE00008301CC008A0192019401210223022433
:1060FE00022502260227022A02B300B4006F0070A6
:10610E000081828330313233919293969734366682
:10611E0067F7F6F53790F0F1F40001E200E900EAD6
:10612E0000B500B600B700CD008301CC008A019205
:10613E000194012102230224022502260227022AAB
:10614E0002B300B4006F00700081828340BC22CF86
:0C615E00091309F1089608AF08C80800F2
:00000001FF
